:020000040000FA
:04000000A9EF00F074
:02000800B8D06E
:0800180006D1076E010E016E16
:100020000850065C02E10750055C040ED8B0010ED2
:10003000D8B4020E0114D8A4010E12000D6E960E53
:10004000056E980E066E55D8D8B4CA90D8A4CA804A
:10005000FC0FD8A0CA92D8B0CA82800E056E960E48
:10006000066E980E096E0A6ACAB025D8CAB223D89D
:1000700042D80504CB6E05C007F006C008F000505A
:100080000B6E0C6E003C0C6A4BD80A500D2E0AD039
:10009000BE6E0C0EBD6E09BEBD8A09BCBD889394B0
:1000A000CA841200BB6E0C0EBA6E09BEBA8A09BCB5
:1000B000BA889492F5D700D8D89009320632053222
:1000C0001200086A076EFF0E0726082200D0D8A08B
:1000D0001200030E066EE70E02D8F5D7066AFE0F71
:1000E000056EE86A065AD8A012000000050600D086
:1000F000F8D70A6A096A100EF36E063409360A3612
:100100000750095C08500A5805E30750095E08507B
:100110000A5AD88005360636F32EEFD7055012005E
:1001200007500B02F3CF09F0F4CF0AF008500B028E
:10013000F3500A2607500C02F3500A260950120009
:10014000086A6BDF04E008C006F007C005F0055040
:100150001200F86A4F0EAF6E240EAC6E900EAB6EAE
:100160000001C69A440E926EE00E936EC00E946E1D
:10017000070EB46E0F0EC16E9DD09EAA1BD0060E48
:10018000AB1412E1E1CF35F0E2CF36F0372A1EEEA4
:1001900080F03750E126000EE222AECFE7FF35C0F7
:1001A000E1FF36C0E2FF1100AE50AE50AB98AB8815
:1001B00011000AD0F2A408D0F294144A152A817AC8
:1001C000136AD6CF12F0110011003750385C14E0DA
:1001D000382AE9CF05F0EACF06F00EEE80F038506D
:1001E000E926000EEA22EF50056E05C0E9FF06C0C1
:1001F000EAFFD880120004D0E868056ED8A012008B
:100200001200376A386A9D8A9F8AF28EF28C120039
:100210009D9A0EEE80F0000EEE6AE82EFDD7376A4A
:10022000386A9D8A1200F29ED8CF5AFEE8CF5BFE54
:10023000E0CF5CFEE9CF5DFEEACF5EFEE1CF5FFE80
:10024000E2CF60FED9CF61FEDACF62FEF6CF63FE69
:10025000F7CF64FEF5CF65FEF3CF66FEF4CF67FE01
:10026000A6CF68FEF28E0001A192F29E5ACED8FF70
:100270005BCEE8FF5CCEE0FF5DCEE9FF5ECEEAFF3D
:100280005FCEE1FF60CEE2FF61CED9FF62CEDAFF42
:1002900063CEF6FF64CEF7FF65CEF5FF66CEF3FFC3
:1002A00067CEF4FF68CEA6FFF28E10009EA8FED7A0
:1002B000AD6E12008B848B8A8B88939A8A9A929067
:1002C0008990929289920068280E076E260E086E19
:1002D000020EB4DE296A316A326A306AABEC03F08E
:1002E000500E2D6E336A33507F08346E939A8A8A8B
:1002F000320EE7DE939A8A9A276A83DF89DFCD6A16
:10030000F294F28A870ED56EB16AA192A082D08E45
:10031000A292B00EB16E59DF166EBA0E165C07E3EC
:10032000FE0E165C02E32AD102D0186A27D116AE5F
:1003300028D0186A890E165C05E116C018F01968F5
:100340001A681ED0990E165C05E116C018F01B68DD
:100350001C6816D0A90E165C05E116C018F01D68C1
:100360001E680ED0B90E165C05E116C018F01F68A5
:10037000206806D0C90E165C03E116C018F021688B
:10038000FDD0185202E1FAD0F9D0890E185C37E19D
:10039000192803E116C019F030D01D0E195C2CE3AA
:1003A0005A0E195C29E21D0E195C00EE45F0EB5067
:1003B000176E325203E11750315C05E31750315E7E
:1003C000000E325A02D0316A326A2DC00EF00F6A26
:1003D00031C010F032C011F010C005F011C006F0AD
:1003E0003450AEDE106E06C011F010500E261150C3
:1003F0000F2233500E242E6E1968C0D0BFD0990E34
:10040000185CD8A463D01B2803E116C01BF05CD095
:1004100016C01CF01C5231E11D0E1B5C2CE35A0E61
:100420001B5C29E21D0E1B5C00EE45F0EB50176EC5
:10043000325203E11750315C05E31750315E000E74
:10044000325A02D0316A326A2DC00EF00F6A31C0C2
:1004500010F032C011F010C005F011C006F0345099
:100460006FDE106E06C011F010500E2611500F22D4
:1004700033500E242E6E1B6881D01D0E1B5C23E3AF
:100480005A0E1B5C20E21D0E1B5C00EE45F0EB508B
:10049000026E3126000E32222DC00EF00F6A31C0DE
:1004A00010F032C011F010C005F011C006F0345049
:1004B00047DE106E06C011F010500E2611500F22AC
:1004C00033500E242E6E1B6859D058D0A90E185CDC
:1004D00009E11D2803E116C01DF002D016C01EF070
:1004E0004DD04CD0B90E185C0AE11F2803E116C0AC
:1004F0001FF003D016C020F07FD840D03FD0C90EE7
:10050000185C3CE121283AE116C021F0E86A21B0EC
:10051000010E0E6E0F6AE86A21B2010E0E26D8B0E7
:100520000F2AE86A21B4010E0E26D8B00F2A0E5009
:1005300021B6010F226E30521EE1225219E02DC069
:100540000EF00F6A31C010F032C011F010C005F08B
:1005500011C006F03450A0EC00F0106E06C011F08F
:1005600010500E2611500F2233500E242E6E02D042
:1005700033C02EF003D0D8902D342E6E27A21CD07D
:100580003FC025F040C026F043C023F044C024F013
:10059000D6CF12F0D7CF13F02350125C245013584B
:1005A000255014582650155815502618D8B0800AD2
:1005B00002E727928B8405D0010E155C02E3146AD2
:1005C000156A305205E1225202E133C02EF003D009
:1005D000D8902D342E6E2E50FF082F6E2FC000F0B5
:1005E000280E076E260E086E020E1EEC00F093D643
:1005F0001D68120021681200070E1F5C21E120C057
:100600002DF0305219E12DC00EF00F6A31C010F0FC
:1006100032C011F010C005F011C006F03450A0EC4B
:1006200000F0106E06C011F010500E2611500F226F
:1006300033500E242E6E03D0D89020342E6E89D0E5
:10064000420E1F5C15E120520FE1316A326A8B8A3B
:10065000296A276A306A89908992500E2D6E336A12
:1006600033507F08346E03D08B9A2968898071D00B
:10067000430E1F5C23E18B942782D6CF12F0D7CF95
:1006800013F0D00E3B6E070E3C6E3BC002F03CC038
:1006900003F002501224236E03501320246E000E28
:1006A0001420256E000E1520266E25C03FF026C0B2
:1006B00040F023C043F024C044F04BD0440E1F5CF4
:1006C00008E1205203E1306A899202D030688982C1
:1006D00040D0450E1F5C24E120C033F033507F082A
:1006E000346E305219E12DC00EF00F6A31C010F097
:1006F00032C011F010C005F011C006F03450A0EC6B
:1007000000F0106E06C011F010500E2611500F228E
:1007100033500E242E6E03D0D8902D342E6E19D067
:10072000460E1F5C0EE1205202E115D809D0010EE1
:10073000205C02E12FD804D0020E205CD8B44BD844
:1007400008D07B0E1F5C05E1316A326A2D503324DC
:100750002E6E1F6812001D0E176E5A0E175C19E2DE
:100760001D0E175C026E590E0E6E0F6A17500E5E4C
:10077000000E0F5AD8900F320E32D8900F320E3230
:100780000E28046E00EE45F0025004C0EBFF172A5D
:10079000E4E112001D0E176E5A0E175C1BE21D0ECF
:1007A000175C026E590E0E6E0F6A17500E5E000E29
:1007B0000F5A0F320E320F320E320F320E321F0E20
:1007C0000F160E28046E00EE45F0025004C0EBFF39
:1007D000172AE2E112001D0E176E5A0E175C19E27D
:1007E0001D0E175C026E590E0E6E0F6A17500E5ECC
:1007F000000E0F5A040ED8900F320E32E82EFBD79F
:100800000E28046E00EE45F0025004C0EBFF172ADC
:06081000E4E11200FFD735
:020000040030CA
:0300010006170ED1
:020005008580F4
:060008000FC00FE00F40E5
:00000001FF
